:0300000002383291
:0C38320078FFE4F6D8FD75816702387954
:102047000A53746172743A20004950436F6E6E658B
:1020570063745245510A00444843502D4F4B0A00C0
:102067004950436F6E6E65637400C0E4E0EFF2E5BC
:10207700F020D1E8EDEAEEEC4950284343290A0065
:10208700C2E5F0F1E8FF20495020ECEEE4F3EBFF66
:102097003A20322E3420EEF22032302E31312E32D9
:1020A7003030350A00C4E0F2E020F1EEE7E4E0ED7D
:1020B700E8FF3A20004F6374203131203230303648
:1020C70000200031343A32303A3039000A000A50E1
:1020D700524F473A20202020202020202020202057
:1020E70020202020202020202020202020202020E9
:1020F70020202020202020202020202020202020D9
:1021070020202020202020202020202020202020C8
:102117002020202020202020200A0044756D7058A0
:102127002020202020303020303120303220303322
:1021370020303420303520303620303720303820DA
:102147003039203041203042203043203044203085
:10215700452030460A003A200044756D704420201F
:1021670020202030302030312030322030332030D2
:102177003420303520303620303720303820303981
:102187002030412030422030432030442030452049
:1021970030460A00457272206B65790052642065EB
:1021A7006570726F6D0A005264204D454D0A0044F8
:1021B700656275674950204F4E0A0044656275672E
:1021C7004950204F46460A00446562756755736556
:1021D70072204F6E0A0044656275675573657220F9
:1021E7004F46460A0044656275674D7367204F6E18
:1021F7000A0044656275674D7367204F46460A00BB
:10220700436F6E666967206C6F636B210A005772B4
:1022170020656570726F6D0A0020536176652065D1
:102227006570726F6D210A00457272204D4143211E
:10223700004C6F61643E3E00576169745265737468
:1022470061727421004E4F4950004C494E4B434F29
:102257004E5452005452415353004652004E4F4C75
:10226700494E4B00494E490000FF224CFF2251FFC7
:0E227700225BFF2261FF2264FF226BFF226FB9
:06401D00010B0001090087
:103FDB00C2AFC28E758900438910758BFF758DB783
:073FEB00D2ABD28ED2AF224F
:03001B0002379C0D
:10379C00C0E0C083C082C0D0C2AFC28E758BFF7533
:1037AC008DB720170675A61E75A6E10509D213E57F
:1037BC000B6002050B050EE50E540F7053D21EE57F
:1037CC000E543F7014D211907A83E0600C04F0E038
:1037DC00D394B44004C2AF80FE907A7EE0600204C1
:1037EC00F0E50AD394014002150A90757BE0600263
:1037FC0014F0907A84E0D394014003E014F0301676
:10380C0002050CE50DD394644004D2178002050D1B
:10381C00E508D3940140021508D28ED2AFD0D0D097
:06382C0082D083D0E032DF
:103E6000E4FFFEFD74512DF582E43477F583E02FF5
:103E7000FFE43EFE0DBD10ECE4FD74A62DF582E4DA
:103E80003475F583E0FC2FFFE43EFEEC60040DBDCD
:023E900080E8C8
:013E9200220D
:10002600C291C290C2B5C21B7D027C007F07123FFF
:10003600888F55E555646060097D017F60123F2316
:10004600D21BE4FDFC7F0B123F888F55E55530E649
:10005600097D04E4FF123F47D21B7D017C007F0728
:10006600123F888F55E5557008FD7FFF123F23D25A
:100076001B301B03126000C2AFC288D2A8C2AA12EC
:100086003AC8C291D290D2AF123E601226C6D2B5FD
:10009600D291C290907A7F121E6C00000000E47F1D
:1000A600207E4EFDFC907A7FE0F8A3E0F9A3E0FA0B
:1000B600A3E0FBC3121E395027907A7FE0FCA3E031
:1000C600FDA3E0FEA3E0FFE4FAF9F8EF2401FFEA5E
:1000D6003EFEE93DFDE83CFC907A7F121E6080BE44
:1000E600D291D2901234DEC217C291D290123D291B
:1000F600D291C29090774FE0C3940350037403F0FB
:10010600D21DD21CD21BD293201B077E207F471202
:100116003243E490796FF0123FDBC2AF750A01A358
:10012600F0C218C219D2AF75A70775A61E75A6E14B
:10013600123FA5D291D290907A7F121E6C000000D9
:1001460000E47F207E4EFDFC907A7FE0F8A3E0F984
:10015600A3E0FAA3E0FBC3121E395027907A7FE092
:10016600FCA3E0FDA3E0FEA3E0FFE4FAF9F8EF2428
:1001760001FFEA3EFEE93DFDE83CFC907A7F121E57
:100186006080BEC291C290201B19AF557E007D03D0
:10019600123328E4FF1235B27E777F6FE4FB7D01D0
:1001A600123406907A83E060037401F0E490757B64
:1001B600F0A37455F0A37481F0E4F50CE4F50D900A
:1001C600757BE070031224B2907A84E0B40111903A
:1001D60080007410F0E4907A84F0D21BD21CD21DF9
:1001E600E50CD39403402D908002E4F0908001F05A
:1001F600908000F0E50CD3940540037401F0E50C03
:10020600D3940A400FE4F50CC214907970F0750A85
:1002160001123D299080A0E070077FCB7E03123942
:10022600C89080B8E070031236609080D0E07014F9
:10023600301F11907A7A74FFF0907743E0FEA3E0C6
:10024600FF123B3D908000E07013301810123137DA
:1002560090772BEFF0D394004003120F4C9080025E
:10026600E07006908000E06005D2160201C2C21658
:10027600E4F50C90757BE060030201C2301A15129A
:100286002D7A90772BEFF0D394004008301205E0DA
:10029600FF123FF22019030204A1122BFD90772BC7
:1002A600EFF070030201C2907A83E060037401F0FC
:1002B60090776FE054BF247F7003020375147003B8
:1002C6000203562402600302044C201B077E207F93
:1002D60050123243907747E0FF700690774BE0600C
:1002E60055907A7AE0FEB50722A3E0FF907748E0C2
:1002F600B50718907A7CE0FF907749E0B5070C9037
:100306007A7DE0FF90774AE06F602B90774BE06E46
:100316007035907A7BE0FF90774CE0B50729907AAC
:100326007CE0FF90774DE0B5071D907A7DE0FF9069
:10033600774EE0B50711C2149079707403F012007D
:1003460021750A010204A1907A7A74FFF00204A1D1
:10035600907A72E0FF907771E06F60030204A190DB
:100366007A72E004F0E4F50A90796FF00204A130A5
:1003760014030204A1907770E0D3940A5003020498
:100386001FA3E06402600302041F907738E0FF9029
:10039600777AE06F60030201C2907739E0FF9077C9
:1003A6007BE06F60030201C290773AE0FF90777CB2
:1003B600E06F60030201C290773BE0FF90777DE03B
:1003C6006F60030201C290773CE0FF90777EE06F9A
:1003D60060030201C290773DE0FF90777FE06F6097
:1003E600030201C27E207F5E12324390777263A2BF
:1003F6000190773063A2017F12122982907784637D
:10040600A201907A7A63A2017F0412298290797000
:100416007406F0750A020201C2743E447770030244
:1004260001C2124024D214E4F50A90796FF0907A52
:100436007E04F0E4907A71F0A3F0201B5E7E207FAC
:1004460067123243805530145290776FE020E74BA5
:10045600907771E0FF907A71E0FE6F600D907A7987
:10046600E07007EE146F70338013907A71E004F039
:1004760090772BE0FFD394044003123E2C907477C0
:100486007482F0A37401F0907771E0907479F07E35
:10049600747F777D03123A490201C22014030205D4
:1004A6005D9080D0E0700B907743E0FEA3E0FF12F2
:1004B6003B3DE50A7066907A7EE0D3943C403790E7
:1004C6007A79E07031120006907A7E7401F0E49039
:1004D600786FF0A37412F0907A72E0907871F0A3BE
:1004E60074FDF090757E63A20190787363A2017F1C
:1004F600121229828006123E93EF60207E787F6F6B
:10050600907870E02404FD123A49907A79E060030D
:100516000201C290774FE0F50A0201C2124001EFD4
:1005260060159074777483F0E4A3F07E747F777D12
:1005360002123A490201C2E50A640160030201C2DD
:1005460090796FE004F0E0C3940540B0C214E4A3D0
:10055600F01200210201C2E50A640160030201C231
:10056600907970E014700302060114700302062DE0
:100576001470030206D514700302078B24FE60690B
:10058600240660030201C2E4F50CF55574272555CF
:10059600F582E43476F583E0FF74302555F582E480
:1005A6003477F583EFF00555E555B43FDF201F217D
:1005B60090774763A201907A7A63A2017F04122999
:1005C600829079707401F090796FF0750A030201D8
:1005D600C29079707404F090796F7401F0750A1402
:1005E600907A7A74FFF00201C2E4F50C123D29906C
:1005F60079707401F0750A030201C2907A7AE0609C
:100606000B907743E0FEA3E0FF123B3D750A029094
:1006160079707402F090773EE070030201C290791F
:10062600707403F00201C2907A7AE070030206C683
:1006360090786F7480F09078717402F0E4A3F0A360
:1006460004F090773863A20190787463A2017F0A60
:1006560012298290787E7430F0A3747BF0E4F5550D
:1006660074A62555F582E43475F583E0FF601174B0
:10067600802555F582E43478F583EFF0055580E062
:1006860074802555F582E43478F583747DF07481A1
:100696002555F582E43478F583E4F0E55524119088
:1006A6007870F07C7A7D7A907743E0FAA3E0FB7F5E
:1006B600021239447E787F6FE5552413FD123A49BC
:1006C6009079707404F090774FE0F50A0201C290B9
:1006D6007A7AE0700302077C90786F7480F09078E5
:1006E600717401F0E4A3F0A304F0A37430F0A374D2
:1006F6007BF0E4F55574A62555F582E43475F5834B
:10070600E0FF601174762555F582E43478F583EFC1
:10071600F0055580E074762555F582E43478F58346
:10072600747DF074772555F582E43478F583E4F02A
:10073600E5552407907870F07C7A7D7A907743E0CF
:10074600FAA3E0FB7F021239447E787F6FE55524D9
:1007560009FD123A49907A79E0601B124024D214BE
:10076600E4F50A90796FF0907A7E04F0E4907A715D
:10077600F0A3F00201C29079707404F090774FE014
:10078600F50A0201C2907A7AE0FF6009F4600690E9
:1007960080027410F0201F2B750A0290796FE064B6
:1007A60001FFF0A37401F0EF600590774780039096
:1007B600774B63A201907A7A63A2017F04122982A1
:1007C6000201C2750A14907A7A74FFF00201C2809F
:0107D600FE24
:0107D70022FF
:100F4C00907770E0B444047F0180027F0090776F4B
:100F5C00E0B447047E0180027E00EE5F604A907729
:100F6C0038E0907771F0907739E0907772F0907765
:100F7C003AE0907773F090773BE0907774F090774D
:100F8C003CE0907775F090773DE0907776F0907735
:100F9C00707452F090772563A2019080A863A2012F
:100FAC007F0612298202145A90772BE0C3940850C2
:100FBC0003021463907738E0FF907771E06F600361
:100FCC00021463907739E0FF907772E06F60030250
:100FDC00146390773AE0FF907773E06F600302142C
:100FEC006390773BE0FF907774E06F6003021463CB
:100FFC0090773CE0FF907775E06F6003021463908C
:10100C00773DE0FF907776E06F6003021463907A8F
:10101C0083E060037401F0907A847464F0907770CC
:10102C007452F090776FE0644D703C7E207F7112AB
:10103C0032437E207F871232431240157E207FACD4
:10104C001232437E207FBC1232437E207FC8123284
:10105C00437E207FCA1232437E207FD31232437EDE
:10106C00207FD51232432290776FE0644C70527E11
:10107C00217F22123243907777E0F556A3E0F557A3
:10108C00E4F5587D03AF57AE561233287E217F5DB1
:10109C00123243AE56AF57E4FB7D101234067E205D
:1010AC007FD312324374102557F557E43556F55655
:1010BC000558E558C3941040CA7E207FD3123243A2
:1010CC002290776FE0646C705CF55A7E217F601221
:1010DC003243E4F559AF5A7E007D031233287E214A
:1010EC007F5D123243E4F558A85AE6FF747925580F
:1010FC00F582E43477F583EFF0055A0558E558B4DA
:10110C0010E67E777F79E4FB7D101234067E207F1B
:10111C00D31232430559E559C3940840B87E207F59
:10112C00D31232432290776FE0644B7046F55874BB
:10113C00612558F582E43477F583E0FF6016747707
:10114C002558F582E43477F583E0B507100558E5AA
:10115C0058B408DB90757B7432F002145A90776F98
:10116C007421F0301B0302145A7E217F9B123243F0
:10117C0002145A90776FE06452704E201B077E2148
:10118C007FA3123243907778E090772BF0E4F558F8
:10119C0090772BE0FDE558C39D5022907777E025A2
:1011AC00582426F582E43476F583E0FF74792558CB
:1011BC00F582E43477F583EFF0055880D37E777FA2
:1011CC006FED240AFD1238BE2290776FE0644970EF
:1011DC0045201B077E217FAE123243907777E0F5D6
:1011EC0056A3E0F557E4F558855782855683E0FF02
:1011FC0074792558F582E43477F583EFF00557E5DB
:10120C0057700205560558E558B480DC7E777F6F21
:10121C007D8A1238BE2290776FE06444600302121C
:10122C00B3907777E0FF6444700302145AEFB43143
:10123C000CC21B7E217FB612324302145A90777770
:10124C00E0B4300CD21B7E217FC212324302145AFE
:10125C00907777E0B4320CD21C7E217FCF123243D0
:10126C0002145A907777E0B4330CC21C7E217FDDD8
:10127C0012324302145A907777E0B4340CD21D7EAC
:10128C00217FEC12324302145A907777E0B4350C7C
:10129C00C21D7E217FF912324302145A907777E0F7
:1012AC00FF12001E02145A90757BE07013201B076E
:1012BC007E227F0712324390776F7421F002145A0A
:1012CC0090757B7432F090776FE0FFB45104C2AF2D
:1012DC0080FEEF64577045201B077E227F1512326B
:1012EC0043907778E090772BF0E4F55890772BE0EB
:1012FC00FFE558C39F400302145A74792558F582B0
:10130C00E43477F583E0FF907777E025582426F5D1
:10131C0082E43476F583EFF0055880D090776FE057
:10132C00645360030213D5201B077E227F201232E8
:10133C0043907738E0FF90762FE06F703C907739D0
:10134C00E0FF907630E06F703090773AE0FF907667
:10135C0031E0B5072490773BE0FF907632E0B5079B
:10136C001890773CE0FF907633E0B5070C90773D12
:10137C00E0FF907634E06F601690776F7421F03058
:10138C001B0302145A7E227F2F12324302145AE49A
:10139C00F558E4F50D74262558F582E43476F5837A
:1013AC00E0FDAF58123FC10558E558C394FE40E22A
:1013BC00C2AFE4907FF0F0A3F0907FFD74AAF0A38D
:1013CC0074FFF0A37455F080FE90776FE0644F705B
:1013DC004B907777E0F556A3E0F557E557455670F7
:1013EC000A201B077E227F38123243201B077F2ADC
:1013FC007E00123243E4F55874792558F582E434B2
:10140C0077F583E0855782855683F00557E557704D
:10141C000205560558E558B480DE803290776FE0AF
:10142C00B4452B201B077E227F3F123243907777E7
:10143C00E0FFA3E0907FF0CFF0A3EFF0C2AF907F7E
:10144C00FD74AAF0A374FFF0A37455F080FE7E77B0
:07145C007F6F7D081238BE0E
:011463002266
:103DF400AE07EEC39430400BEED394395005EE2455
:103E0400D0FF22EEC39461400BEED394665005EECE
:103E140024A9FF22EEC39441400BEED394465005EF
:083E2400EE24C9FF22AF0622C3
:1026C600C212E4907A83F0D21FC215907A79F09004
:1026D600773863A201907A7363A2017F061229827A
:1026E600E4F556E55675F003A42470F582E4342229
:1026F600F583E493FB740193FA740293F9121D01B6
:1027060070030228A6E4F557F558FD74A62DF58248
:10271600E43475F583E0FF70030228A1E55675F0F1
:1027260003A42470F582E43422F583E493FB740158
:1027360093FA740293F9855782758300121D1AFE67
:10274600EFB50608755801055702289DE558700330
:1027560002289DEE6003022898E55624FE602214A6
:10276600700302288814700302288C147003022850
:1027760094240460030228A1907A837401F002284D
:10278600A1D21274A62DF582E43475F583E0FF64B8
:102796002D70030228A1123DF4EFC454F0FC74A777
:1027A6002DF582E43475F583E0FF123DF4EF2C90AD
:1027B6007A73F074A82DF582E43475F583E0FF1280
:1027C6003DF4EFC454F0FC74A92DF582E43475F59C
:1027D60083E0FF123DF4EF2C907A74F074AA2DF585
:1027E60082E43475F583E0FF123DF4EFC454F0FC47
:1027F60074AB2DF582E43475F583E0FF123DF4EFFA
:102806002C907A75F074AC2DF582E43475F583E07E
:10281600FF123DF4EFC454F0FC74AD2DF582E434A0
:1028260075F583E0FF123DF4EF2C907A76F074AEE6
:102836002DF582E43475F583E0FF123DF4EFC454C0
:10284600F0FC74AF2DF582E43475F583E0FF123D9C
:10285600F4EF2C907A77F074B02DF582E43475F5A8
:1028660083E0FF123DF4EFC454F0FC74B12DF58201
:10287600E43475F583E0FF123DF4EF2C907A78F09E
:102886008019D2158015907A797401F0800DC21FD7
:102896008009E4F558F5570D02271105560226E979
:0128A600220F
:03000300023C6C50
:0D3C6C00C0E0C083C082C0D075D000C0078A
:103C7900C2A8908008E0FFEF54F06035EF30E40807
:103C8900D2189080087410F0EF30E508D21A9080AD
:103C9900087420F0EF30E608D2199080087440F0DB
:103CA900EF30E7069080087480F0908008E0FF808C
:093CB900C690800874FFF0D2A847
:0B3CC200D007D0D0D082D083D0E032F9
:103D29009080007480F090773063A201F583F5826A
:103D390063A2017F0812298290773863A2019080DB
:103D49008863A2017F0A122982907742E0FF90805E
:103D5900B1F09080E1EFF09080957455F0A3F09068
:0C3D690080007401F09080097470F0225A
:0439C800AD07AC0695
:1039CC00908009E04410F09080A0E0706F9080A18E
:1039DC007482F09080A874FFF0A3F0A3F0A3F0AF72
:1039EC0004AE079080AEEEF0AE05A3EEF0AE0790FD
:1039FC0080ACEEF0AE05A3EEF09080007402F09077
:103A0C007BA3121E6C00000000907BA3E090804012
:103A1C00F0907BA4E0908041F0907BA5E0908042F8
:103A2C00F0907BA6E0908043F0A3E4F0A3F0A3F029
:0C3A3C00A3F0908018F0A3F0A3F0A3F01A
:013A4800225B
:043B3D00AD07AC061E
:103B4100908009E04440F09080D0E070559080D1A1
:103B51007482F0AF049080DEEFF0AF05A3EFF09038
:103B610080027402F0907BA7121E6C00000000908E
:103B71007BA7E0908058F0907BA8E0908059F0906E
:103B81007BA9E090805AF0907BAAE090805BF0A343
:103B9100E4F0A3F0A3F0A3F0908030F0A3F0A3F041
:023BA100A3F08F
:013BA30022FF
:10366000908009E04420F09080B8E06003023701C8
:103670009080B97482F07F039080C6EFF07FCDA375
:10368000EFF07F039080C4EFF0A374CDF030002200
:10369000907747E09080C0F0907748E09080C1F04C
:1036A000907749E09080C2F090774AE09080C3F034
:1036B000800C9080C074FFF0A3F0A3F0A3F0908082
:1036C000017402F0907BAB121E6C00000000907B36
:1036D000A7E090804CF0907BA8E090804DF0907B2C
:1036E000A9E090804EF0907BAAE090804FF0A3E498
:1036F000F0A3F0A3F0A3F0908024F0A3F0A3F0A334
:01370000F0D8
:0137010022A5
:103944008C568D57A907EAFDE975F018A424ACFF3D
:10395400E5F034808F82F583EDF0EBFDE975F01826
:10396400A4FFAEF024ACFBEE34808B82F583A3ED90
:10397400F08557828C83E0FDEF24A8FFEE3480FEAF
:103984008F82F583EDF08557828C83A3E08F828E3E
:1039940083A3F0855782855683A3A3E0FDE975F0E0
:1039A40018A424A8FFE5F03480FE8F82F583A3A336
:1039B400EDF08557828C83A3A3A3E08F828E83A32B
:0439C400A3A3F022A7
:0638BE008D5BAB07AA06BA
:1038C400907BA3E0FCA3E0FDA3E0FEA3E0F55F8E04
:1038D4005E8D5D8C5CAE02AF038E838F8263A2012A
:1038E400E55E540744C0F583855F8263A201AF5B44
:1038F4001229EB908000E020E5F9E4FCFDFEE55F91
:10390400255BF55FEE355EF55EED355DF55DEC3519
:103914005CF55CC2A8908040E55CF0A3E55DF0A393
:10392400E55EF0A3E55FF0D2A89080007420F0AFCC
:0F3934005FAE5EAD5DAC5C907BA3121E60AF5BBF
:013943002261
:063A49008D56AB07AA0632
:103A4F00907BA7E0FCA3E0FDA3E0FEA3E0F55A8E78
:103A5F00598D588C57AE02AF038E838F8263A201AC
:103A6F00E559540744D0F583855A8263A201AF56B6
:103A7F001229EBE4FCFDFEE55A2556F55AEE3559B1
:103A8F00F559ED3558F558EC3557F557C2A89080D4
:103A9F0058E557F0A3E558F0A3E559F0A3E55AF020
:103AAF00D2A89080027420F0AF5AAE59AD58AC57DF
:083ABF00907BA7121E60AF56B8
:013AC70022DC
:0235B2008F5731
:1035B400908001E030E5037F0022907BABE0FCA328
:1035C400E0FDA3E0FEA3E0F55B8E5A8D598C589084
:1035D4007A7363A201E55A540744C8F583855B8274
:1035E40063A2017F06122A01E55B2406F55BE4353C
:1035F4005AF55AE43559F559E43558F55890797126
:1036040063A201E55A540744C8F583855B8263A22B
:1036140001AF57122A01E4FCFDFEE55B2557F55B7B
:10362400EE355AF55AED3559F559EC3558F558C279
:10363400A890804CE558F0A3E559F0A3E55AF0A30F
:10364400E55BF0D2A89080017420F0AF5BAE5AAD78
:0B36540059AC58907BAB121E60AF57C2
:01365F002248
:10313700C2A89081E0E0F556055605560556055696
:10314700055605560556055605560556908010E056
:10315700F559A3E0F55AA3E0F55BA3E0F55C908190
:10316700E1E0F5560556055605560556055605562A
:103177000556055605560556908014E0F55DA3E003
:10318700F55EA3E0F55FA3E0F560D2A8E55FB55B68
:1031970008E560B55C037F0022E4F556E55F540758
:1031A70044E0F58385608263A20190776F63A20193
:1031B7007F08122A1990777163A20190772563A27D
:1031C700017F0612298290776FE0F557A3E0F55843
:1031D700E4F55690776FE0702AA3E024F8F556E5FA
:1031E7005F540744E0F58385608274082582F58281
:1031F700E43583F58363A20190776F63A201AF562D
:10320700122A19AE57E4FCFDE5602558F560E55F25
:103217003EF55FED355EF55EEC355DF55DC2A89078
:103227008014E55DF0A3E55EF0A3E55FF0A3E5603C
:0B323700F0D2A89080007440F0AF5669
:013242002269
:102BFD00C2A89081E6E0F5560556055605560556D0
:102C0D00055605560556055605560556908028E07D
:102C1D00F559A3E0F55AA3E0F55BA3E0F55C9081CF
:102C2D00E7E0F55605560556055605560556055663
:102C3D00055605560556055690802CE0F55DA3E02A
:102C4D00F55EA3E0F55FA3E0F560D2A8E4F556E5E7
:102C5D005FB55B0AE560B55C05C219022D5BE55FEA
:102C6D00540744F0F58385608263A20190776F630A
:102C7D00A2017F08122A1990776FE0F557A3E0F5AE
:102C8D0058E558455770099080027410F07F002266
:102C9D00907A7AE0FFF4602D907771E06F70769006
:102CAD007A7BE0FF907772E06F706A907A7CE0FF3C
:102CBD00907773E06F705E907A7DE0FF907774E0AF
:102CCD006F60228050907771E0907A7AF0907772F1
:102CDD00E0907A7BF0907773E0907A7CF090777447
:102CED00E0907A7DF090776FE0702AA3E024F8F5FC
:102CFD0056E55F540744F0F583856082740825829C
:102D0D00F582E43583F58363A20190776F63A201A9
:102D1D00AF56122A19AE57E4FCFDE5602558F56053
:102D2D00E55F3EF55FED355EF55EEC355DF55DAF6E
:102D3D005CAE5BAD5AAC59AB60AA5FA95EA85DD322
:102D4D00121E4F40099080027410F07F0022C2A81D
:102D5D0090802CE55DF0A3E55EF0A3E55FF0A3E5C3
:0C2D6D0060F0D2A89080027440F0AF56D5
:012D79002237
:102D7A00C2A89081E3E0F556055605560556055654
:102D8A0005560556055605560556055690801CE00B
:102D9A00F559A3E0F55AA3E0F55BA3E0F55C908151
:102DAA00E4E0F556055605560556055605560556E8
:102DBA000556055605560556908020E0F55DA3E0B8
:102DCA00F55EA3E0F55FA3E0F560D2A8E4F556E569
:102DDA005FB55B0AE560B55C05C21A022EC2E55F03
:102DEA00540744E8F58385608263A20190747B638B
:102DFA00A2017F0E122A2F90747BE0F557A3E0F50B
:102E0A0058907A73E0FF907483E06F706C907A74D4
:102E1A00E0FF907484E06F7060907A75E0FF9074C0
:102E2A0085E06F7054907A76E0FF907486E06F7058
:102E3A0048907A77E0FF907487E06F703C907A78D8
:102E4A00E0FF907488E06F703090747BE0702AA382
:102E5A00E024F2F556E55F540744E8F5838560827D
:102E6A00740E2582F582E43583F58363A20190749A
:102E7A007B63A201AF56122A2FAE57E4FCFDE56030
:102E8A002558F560E55F3EF55FED355EF55EEC359C
:102E9A005DF55DAF5CAE5BAD5AAC59AB60AA5FA99C
:102EAA005EA85DD3121E4F5006E55845577009902B
:102EBA0080017410F07F0022C2A8908020E55DF0A6
:102ECA00A3E55EF0A3E55FF0A3E560F0D2A89080E9
:062EDA00017440F0AF5648
:012EE00022CF
:043243008E5B8F5CB3
:10324700907BA3E0FCA3E0FDA3E0FEA3E0F5628E84
:10325700618D608C5FE562FFE5615407FEE42FF541
:103267005EEE34C0F55D855E82F5837423F0055EFE
:10327700E55E7002055D535DC7F582855D83740A5F
:10328700F0055EE55E7002055D535DC790773863B4
:10329700A201855D83855E8263A2017F061229EB09
:1032A7007406255EF55EE4355DF55D855B83855CBB
:1032B7008263A201855D83855E8263A2011229CFA5
:1032C700908000E020E5F9E4FCFDFE907BA3E0F8A8
:1032D700A3E0F9A3E0FAA3E02FFFEE3AFEED39FDF4
:1032E700EC38FCEF2408FFE43EFEE43DFDE43CFC43
:1032F700907BA3121E60C2A8907BA3E0908040F051
:10330700907BA4E0908041F0907BA5E0908042F014
:10331700907BA6E0908043F0D2A89080007420F0C4
:013327002283
:063406008E5B8F5C8D5D02
:10340C00907BA3E0FCA3E0FDA3E0FEA3E0F5638EBC
:10341C00628D618C60E563FFE5625407FEE42FF575
:10342C005FEE34C0F55E855F82F5837423F0055F33
:10343C00E55F7002055E535EC7F582855E83EBF037
:10344C00055FE55F7002055E535EC790773863A237
:10345C0001855E83855F8263A2017F061229EB746E
:10346C0006255FF55FE4355EF55E855B83855C82E2
:10347C0063A201855E83855F8263A201AF5D122921
:10348C00EB908000E020E5F97408255DF55DFFE424
:10349C00FCFDFEE5632FF563EE3562F562ED3561FB
:1034AC00F561EC3560F560C2A8908040E560F0A352
:1034BC00E561F0A3E562F0A3E563F0D2A89080008B
:1034CC007420F0AF63AE62AD61AC60907BA3121E52
:0134DC00608F
:0134DD0022CC
:063328008E5B8F5CAB051B
:10332E00907BA3E0FCA3E0FDA3E0FEA3E0F5628E9C
:10333E00618D608C5FE562FFE5615407FEE42FF559
:10334E005EEE34C0F55D855E82F5837423F0055E16
:10335E00E55E7002055D535DC7F582855D83EBF01A
:10336E00055EE55E7002055D90773863A201855DAE
:10337E0083855E8263A2017F061229EB7406255EA9
:10338E00F55EE4355DF55D535DC7E55B855E828573
:10339E005D83F0055EE55E7002055D535DC7F582E7
:1033AE00855D83E55CF0055EE55E7002055D535D4F
:1033BE00C7908000E020E5F9E562240AF562E43565
:1033CE0061F561E43560F560E4355FF55FC2A890A4
:1033DE008040E55FF0A3E560F0A3E561F0A3E56250
:1033EE00F0D2A89080007420F0AF62AE61AD60ACF8
:0733FE005F907BA3121E602B
:0134050022A4
:103F6B00E5D220E0FBC2AF438E2075D2028F827563
:0C3F7B008300E0FFE4F5D2538EDFD2AFEC
:013F87002217
:103FC100E5D220E0FBC2AF43D2028F82758300EDC0
:0A3FD100F075D25063D250D2AF2237
:103AC800E4FEEE04FF123F6B74302EF582E4347787
:103AD800F583EFF00EBE3FEAE4FEEE247FFF123FCF
:103AE8006B74A62EF582E43475F583EFF074A62E78
:103AF800F582E43475F583E0701B74A62EF582E434
:103B08003475F5837420F074A72EF582E43475F5C6
:103B180083E4F080040EBE80C1E4907625F0FEAF09
:103B280006123F6B74262EF582E43476F583EFF0A7
:043B38000EBEFEEBD4
:013B3C002266
:103F8800A2AF9225C2AF8C838D82EF122A4743A23B
:0C3F980020122A4953A2DFA22592AFFF9D
:013FA40022FA
:023F23008F56B7
:103F2500A2AF9225C2AFE4F5838D827406122A47AB
:103F3500E55643A220122A4953A2DFA22592AF7F5C
:013F4500017A
:013F46002258
:023F47008F5693
:103F4900A2AF9225C2AFE4F5838D82740A122A4783
:103F5900E55643A220122A4953A2DFA22592AF7F38
:013F69000156
:013F6A002234
:1028A700A907E7FFA805EF93C3966008403B74FCB0
:1028B7002FFF80F00F08EF93C3966008402B74FB3F
:1028C7002FFF80E00F08EF93C3966008401B74FA50
:1028D7002FFF80D00F08EF93D3966008400B74F951
:1028E7002FFF80C01F1F1F1F1FEF54FEF80303F7A2
:1028F700E893FC08E893FD08E893FE08E893FF22B5
:1029070009E993C39D6008402974FB29F980F109FF
:10291700E993C39E6008401A74FA29F980E209E92D
:1029270093D39F6008400B74F929F980D3191919BB
:102937001919E9C313C313FF22740093F8ECC39862
:102947004024701F740193F8EDC3984019701474F4
:0E2957000293F8EEC398400E7009740393F8D3
:10296500EFC39840037F00227F0122EDF8E6F008CF
:10297500A3DFFA22EDF8E0F608A3DFFA22E0A3636D
:10298500A201F0A363A201DFF475A20022E0A36314
:10299500A201F0A363A201E0A363A201F0A363A2D5
:1029A50001E463A201F0A363A201DFE175A20022A5
:1029B500E0A363A2016DFE936CFDEE058393FC1508
:1029C5008363A201DFEA75A200227F00E493A3637B
:1029D500A201F00F600CA3E583C2E3F58363A201B6
:1029E50080EA75A20022E0A363A201F0A3E583C2F9
:1029F500E3F58363A201DFEE75A20022E0A363A2E3
:102A050001F0A3E583C2E4D2E3F58363A201DFEC21
:102A150075A20022E583C2E3F583E0A363A201F07A
:102A2500A363A201DFEE75A20022E583C2E4D2E32F
:102A3500F583E0A363A201F0A363A201DFEC75A215
:102A45000022F922C002C004C00612FFF0D006D051
:042A550004D0022285
:103D750020536572763A0020547261737353656EF1
:103D8500644552520A00205265496E6974204341C8
:103D95004E0A002043414E283029203E20544F2111
:103DA5000A0020545520300A0020545520310A00BD
:03001E00E4FF22DA
:103EC600C28DC2AF438901C28C907A99E0FF700718
:103ED600F58A758CEE8016EFB40508E4F58A758CC4
:103EE600B8800AEFB40A06E4F58A758C70D28CD2D3
:023EF600AF22F9
:103DB500C28DC2AF438901C28C907A99E0FF70141D
:103DC500302409F58A758CDCC224801E758A6675D7
:103DD5008CFC8016EFB40508E4F58A758CEE800A34
:0F3DE500EFB40A06E4F58A758CDCD28CD2AF22DB
:103FA500123BA4120022D223E4F550907BA1F0F538
:0C3FB5003EF554123EC6C224E4F5522230
:103E2C00EF24FCF556201B127E3D7F751232437E2B
:103E3C00777F737B01AD5612340690777363A201C2
:103E4C00907B2163A201AF5612298285563EE4F580
:033E5C004FC22131
:013E5F002240
:0F3FF200D3EF6480948E5006E55470028F5422F2
:1024B200208D0302254EC28C2023030225A7E53E70
:1024C20060547425254FF582E4347BF583E02405BE
:1024D200F556D3940E4008E4F53ED2210225A774A6
:1024E20021254FF582E4347BF5837D40AF561229D6
:1024F20079E556254FF54FE54030E702D224123EEA
:10250200C6123CCDE54FC3953E50030225A7E4F524
:102512003ED2210225A7E5516014907A857D40FFC5
:10252200122979123EC6123CCDE4F5518077E5546A
:10253200601490747B7D40FF122979123EC6123CD2
:10254200CDE4F554805F123C09123EC6122EE18F93
:1025520056EF6051123DB5E4F552E553C3946E5007
:1025620018749A2553F582E4347AF583E556255397
:10257200F5537D40AF56122970301224E54030E702
:102582000330001C9079717D40AF56122970AF560E
:102592001235B2EF700A201B077E3D7F7C12324358
:1025A200AF56123022301E1230110D0552E552D3B1
:1025B20094F04004C2AF80FEC21E2013030226C262
:1025C200906001E004F07006906000E004F0E550D5
:1025D2006031D39401400415508028907BA1E0041F
:1025E200F0E0D39403400D201B077E3D7F8B123217
:1025F20043123FA5201B077E3D7F98123243E4F52C
:1026020050D223302243E551703F907A8504F0A3E3
:102612007408F0A37480F0A37401F0A37406F09020
:102622007B1CE0907A8AF0907B1DE0907A8BF09090
:102632007B1EE0907A8CF0907B1FE0907A8DF0E424
:10264200A3F0A3F075510BC222302072907B1AE0E6
:102652007035E5517031907A857442F0A37408F0B8
:10266200907B1BE0907A87F0907B20E0907A88F054
:10267200A37401F0755106201B077E3D7FA712321D
:1026820043907B1AE004F0907B1AE06402702FE51D
:1026920051702B907A857402F0A37408F0907B1B22
:1026A200E0907A87F0A3F0A37401F0755106201B25
:1026B200077E3D7FAE123243907B1AE004F0C213D4
:0326C2001207D824
:0126C50022F2
:103E9300E553602CE490786FF0A3E553F0907A72C9
:103EA300E0907871F0A37419F0907A9A63A201906C
:103EB300787363A201AF53122982E4F5537F012281
:033EC3007F00225B
:0B400100302105C2217F01227F002238
:0100210022BC
:06402400E4F553F53E2215
:100006007F01E490757EF0A3F0A3F0FEEF25E0FFFC
:040016000EBE08F81A
:01001A0022C3
:103EF8002043616E457247495400200A00204B5602
:103F080054210A002043616E457272434821000A19
:0B3F1800000A20526571457272210002
:102EE100E59B541F6020201B1A7E3E7FF81232435F
:102EF100E59B541FFF7E007D031233287E3F7F0236
:102F0100123243E4F59BE5BA30E010E4F5B375B154
:102F110080F5B2D223F550907BA1F0E5CFF4700398
:102F210002301F755801E4F557E5CFF45558700389
:102F310002300DE557C454F0F5B1E5B2547F642079
:102F41006003022FCFE5B3540FF54485BC40200048
:102F510016E5BD541FFF131313541FFFE5BD54E0C5
:102F610044184FF5418006E5BD54E0F541E5BDC487
:102F71003354E0FFE5BE131313541F4FF542E5BE72
:102F8100C43354E0FFE5BF131313541F4FF54385BA
:102F9100A34585A34685A34785A34885A34985A362
:102FA1004A85A34B85A34CE4F5B230000C85AE4DA8
:102FB10085AF4E75B3D07F0F22E540547EB54005F5
:102FC10075B350800375B3D0E5442405FF22E5B203
:102FD10030E60A201B077E3F7F05123243E5B254DB
:102FE1009F6023201B207E3F7F0C123243AFB27EB5
:102FF100007D03123328AFB37E007D031233287E98
:103001003F7F17123243E4F5B275B3D0E55825E09E
:10301100F5580557E557C394085003022F2A7F003E
:01302100228C
:103CCD0020005875B180E4F5B3F5B28540BCE542EE
:103CDD00C4135407FFE54154E04FF5BDE5423333BE
:103CED003354F8FFE543C41354074FF5BEE5433392
:103CFD00333354F8F5BF8545A38546A38547A38582
:103D0D0048A38549A3854AA3854BA3854CA3E544C8
:0C3D1D00540F2450F5B375500AC2232245
:103C090020005F75B190E5B220E613201B107E3FBE
:103C19007F19123243AFB27E007D03123328E4F5D7
:103C2900B3F5B27497250FF582E43461F583E0F5B5
:103C3900BCE4F5BD7498250FF582E43461F583E0A1
:103C4900FF33333354F8F5BE75BF78050F050F748C
:103C590097250FF582E43461F583E07002F50F755D
:033C6900B3502233
:09400C00EF6003C29622D2962255
:103BA40043AB01C2E8C2EAE4FFEFC454F0F5B1C389
:103BB400EF64809488500575B3D08003E4F5B3E4D2
:103BC400F5B2F5BCF5BDF5BEF5BFF5C4F5C5F5C652
:103BD400F5C7F5A3F5A3F5A3F5A3F5A3F5A3F5A3FD
:103BE400F5A30FBF0EC3907A99E0FF25E0F5B475F5
:103BF400B50C75B66C75A11275AB0275C13E75C373
:043C0400FF75C20383
:013C08002299
:10146400C7E0E3F0F3E7EEF7EDFBE920EEE1F0E0AF
:10147400E73A20CACF20C8F1E5F2FC207620312ECD
:10148400303328C8D1C5D2DC290A005452414E5AFF
:10149400004D415842005254530044454C415900B8
:1014A4004E4F4B5654004B5000424F4F5400434153
:1014B4004E004E4557504B540041540044434400A1
:1014C40043414E4D4F4E0054454C3A004C434C0062
:1014D4004454420054524300000A4F55543A0044C5
:1014E40043445F4F4646210A00446973636F6E6E3E
:1014F4006563746564210A004D4F44454D5F4F4B4D
:10150400210A004D4F44454D5F434F4E4E454354D1
:10151400210A004D4F44454D5F4C495354454E21DB
:101524000A004D4F44454D5F4552524F52210A0027
:101534004D4F44454D5F434F4E4E4543545F4641E6
:10154400494C555245210A004D4F44454D5F44498D
:1015540053434F4E4E4543544544210A005254537D
:101564000A004D6F64656D20696E69740A00CDE5EB
:10157400F220EEF2E2E5F2E0210A004469616C69CE
:101584006E670A00CEF820E4EBE8EDFB210A000ABE
:10159400CDE5F220CAE2E8F2E0EDF6E8E821000A3F
:1015A400436F6E66205265712100CCEEE4E5EC20B9
:1015B400E220F5EE2DF0E5E6E8ECE5210A00C1F0C5
:1015C400E0EAF3E5EC210A000A4352432045525273
:1015D4003A20000A494E3A00436F6E662052656114
:1015E4006479210A00436F6E6620426C6F636B213D
:1015F4000A00CFF0E8EDFFF2FB20E4E0EDEDFBE5BF
:1016040020E1E5E720F1EEE5E4E8EDE5EDE8FF2192
:101614000A000A446174613A20003F3F3F0A000017
:1016240089129B24AD36BF48C15AD36CE57EF7813D
:1016340008931AA52CB73EC940DB52ED64FF76022D
:101644008B109926AF34BD4AC358D16EE77CF5831D
:101654000A9118A72EB53CCB42D950EF66FD74040D
:101664008D169F20A932BB4CC55ED768E17AF385FD
:101674000C971EA128B33ACD44DF56E960FB7206ED
:101684008F149D22AB30B94EC75CD56AE378F187DD
:101694000E951CA32AB138CF46DD54EB62F97008CD
:1016A400811A932CA53EB740C952DB64ED76FF89BD
:1016B400009B12AD24BF36C148D35AE56CF77E0AAD
:1016C4008318912EA73CB542CB50D966EF74FD8B9D
:1016D400029910AF26BD34C34AD158E76EF57C0C8D
:1016E400851E9728A13AB344CD56DF60E972FB8D7D
:1016F400049F16A920BB32C54CD75EE168F37A0E6D
:10170400871C952AA338B146CF54DD62EB70F98F5C
:10171400069D14AB22B930C74ED55CE36AF178005C
:10172400112332465765748C9DAFBECADBE9F810AD
:10173400013322564775649C8DBFAEDACBF9E8219C
:1017440030021367764455ADBC8E9FEBFAC8D9318D
:1017540020120377665445BDAC9E8FFBEAD8C9427C
:1017640053617004152736CEDFEDFC8899ABBA526D
:1017740043716014053726DECFFDEC9889BBAA635C
:1017840072405125340617EFFECCDDA9B88A9B734D
:1017940062504135241607FFEEDCCDB9A89A8B843C
:1017A40095A7B6C2D3E1F008192B3A4E5F6D7C942D
:1017B40085B7A6D2C3F1E018093B2A5E4F7D6CA51C
:1017C400B48697E3F2C0D129380A1B6F7E4C5DB50D
:1017D400A49687F3E2D0C139281A0B7F6E5C4DC6FC
:1017E400D7E5F48091A3B24A5B69780C1D2F3ED6ED
:1017F400C7F5E49081B3A25A4B79681C0D3F2EE7DC
:10180400F6C4D5A1B082936B7A48592D3C0E1FF7CC
:10181400E6D4C5B1A092837B6A58493D2C1E0F7C47
:101824002B2B2B7C0D6174680D7C61747A0D004F39
:101834004B0D0A0000000000000000000000000042
:101844000000004F4B0D0A000000000000000000E3
:1018540000000000000000434F4E4E4543540D0A63
:1018640000000000000000000000004C49535445F3
:101874004E0D0A00000000000000000000000045BA
:1018840052524F520D0A00000000000000000000F8
:10189400000000434F4E4E454354204641494C55A9
:1018A40052450D0A000000444953434F4E4E4543F0
:1018B4005445440D0A000000000000000000000030
:1018C400000000000000000000000000000000FF15
:1018D400148FFF1495FF149AFF149EFF14A4FF1491
:1018E400AAFF14ADFF14B2FF14B6FF14BDFF14C059
:1018F400FF14C4FF14CBFF14D0FF14D4FF14D8FF7B
:0219040014DCF1
:084015007E147F641232432285
:0300230002228531
:0B228500C0E0C083C082C0D075D0183C
:102290002098030223DFC298750B01AF9930010328
:1022A000022362BF020C906192E4F0D201D291024B
:1022B00023DF2010030223DF901847E493B51F1398
:1022C0009061927401F09061957418F0A37448F0D5
:1022D00002235390185BE493B51F1290619274022D
:1022E000F09061957418F0A3745CF0806690186F9C
:1022F000E493B51F129061927403F0906195741885
:10230000F0A37470F0804C901883E493B51F129082
:1023100061927404F09061957418F0A37484F08055
:1023200032901897E493B51F129061927405F09063
:1023300061957418F0A37498F080189018ABE4932A
:10234000B51F109061927406F09061957418F0A317
:1023500074ACF0906192E070030223DFD201D2915D
:10236000807D906192E0FE6044906195E0FCA3E086
:10237000F5828C83E493B51F29906196E004F07098
:1023800006906195E004F0BF0A149061C7EEF0A3D7
:10239000E4F0906192F0C201F52DC2918041052DCB
:1023A000803DC291906192E4F0C2018032300B070F
:1023B000C20B531F0F8019BF0904D20B8021BF032A
:1023C0000F852D38632D80532D80C201C291800F5F
:1023D0007434252DF582E4346FF583EFF0052D205C
:1023E00099030224A92002030224A720090302243E
:1023F0006EE534B4FF0D7599020534753900D2903D
:102400000224A7E534B52C147599030534906F3375
:10241000E070030224A77401F00224A7E534D395E9
:102420002C4008C202D210C290807CE53960133083
:1024300003064420F59980038539990534753900E0
:10244000806574342534F582E43470F583E0F53921
:102450006402600BE53964036005E539B40905756C
:102460009909804385399905347539008039743468
:102470002534F582E43470F583E0FF7008C202D29F
:1024800010C2908022D290C210EFB47C090534753E
:102490000832C2028011AF34053474342FF582E45F
:0924A0003470F583E0F599C2994E
:0924A900D0D0D082D083D0E03203
:10190600C20ED20DC200907134741EF0E4907A9922
:10191600F0C203C204C206C205F536C20AC20CC230
:1019260008906F33F090619774C4F0E4A3F0A37449
:10193600C4F0A37401F0A374C8F0E4A3F0A374C8C0
:10194600F0A37401F0A374C2F0E4A3F0A374C2F090
:10195600A37401F0E4A3F0A3F0F50F907BAFF09031
:101966007BAFE075F003A424D3F582E43418F58345
:10197600E493FB740193FA740293F9121D01700348
:10198600021D00E4907BB1F0A3F0907BB0F0907B59
:10199600B0E024A6F582E43475F583E0FF70030217
:1019A6001CF7907BAFE075F003A424D3F582E434F2
:1019B60018F583E493FB740193FA740293F9907B10
:1019C600B1E0F582758300121D1AFEEFB5060F9081
:1019D6007BB27401F0907BB1E004F0021CEE907BC8
:1019E600B2E07003021CEEEE6003021CE5907BAFD2
:1019F600E0B410004003021CF7901A06F82828737A
:101A0600021A36021A83021CF7021CF7021B9A02FC
:101A16001BD0021BFF021B9F021C04021C09021C96
:101A260057021C5C021C61021CD5021CD9021CDD7B
:101A3600907BB0E024A6F9E43475FA7B01C0031B61
:101A46008B59755A00755B00E4F55CD003122A5970
:101A5600907BB3121E60907BB3E0F8A3E0F9A3E09D
:101A6600FAA3E0FB7F007E8C7D0A7C00121D991292
:101A76001E2B907475EEF0A3EFF0021CF7907BB767
:101A86007461F0A37497F0907BB0E024A6F582E42D
:101A96003475F583E024D0F50FC394014007E50FB4
:101AA600D394084003E4F50FE50F6028907BB7E474
:101AB60075F001121D4785F082F58374C4F0150F89
:101AC600907BB7E475F001121D4785F082F583E53A
:101AD6000FF080D4907BB0E024A7F582E43475F54E
:101AE60083E024D0F50FC394014007E50FD3940893
:101AF6004003E4F50FE50F6028907BB7E475F0012D
:101B0600121D4785F082F58374C8F0150F907BB7D8
:101B1600E475F001121D4785F082F583E50FF0802C
:101B2600D4907BB0E024A8F582E43475F583E024F4
:101B3600D0F50FC394014007E50FD394084003E4A2
:101B4600F50FE50F6028907BB7E475F001121D478D
:101B560085F082F58374C2F0150F907BB7E475F0BB
:101B660001121D4785F082F583E50FF080D4907B46
:101B7600B7E475F001121D4785F082F583E4F09015
:101B86007BB775F001121D4785F082F583E4F0F509
:101B96000F021CF7D208021CF7907BB0E024A6F9CE
:101BA600E43475FA7B01C0031B8B59755A00755BCB
:101BB60000E4F55CD003122A59907BB3121E6090A4
:101BC6007BB6E0907A99F0021CF7907BB0E024A6F1
:101BD600F9E43475FA7B01C0031B8B59755A0075FD
:101BE6005B00E4F55CD003122A59907BB3121E60A9
:101BF600907BB6E0F536021CF7D204021CF7D2033E
:101C0600021CF7907BB0E024A6F9E43475FA7B0158
:101C1600C0031B8B59755A00755B00E4F55CD00355
:101C2600122A59907BB3121E60E4FFFEFDFC907BE6
:101C3600B3E0F8A3E0F9A3E0FAA3E0FBD3121E4F4A
:101C46004008907BB6E0907134F0D20EC20D021CB3
:101C5600F7D206021CF7D200021CF7E4F50F907BC0
:101C6600B0E024A6F582E43475AF82907BB7F0A38A
:101C7600EFF0907BB7E0FEA3E0F5828E83E0FF6491
:101C860020602AEF6027E50FC394255020AE0F058C
:101C96000F74022EF582E43461F583EFF0907BB881
:101CA600E004F07006907BB7E004F080C5AF0F0546
:101CB6000F74022FF582E43461F583740DF074021B
:101CC600250FF582E43461F583E4F0F50F8022D226
:101CD6000A801ED20C801A906F337401F08012E4D1
:101CE600907BB2F0907BB1F0907BB0E004F00219EB
:0A1CF60094907BAFE004F002196542
:011D000022C0
:1034DE00E4F52A9061C8F0C207906193F0906F32C4
:1034EE007405F0C202C210C201C20BE4F534F52C11
:1034FE00F508F52DF50B90747574FFF0A374F4F0C8
:10350E00121906907134E004F528E4F53575F0755E
:10351E00E535A42449F582E5F03468F583E4F0E559
:10352E003575F00DA4242AF582E43461F583E4F0B8
:10353E00F52B75F068E535A42435F582E5F0347188
:10354E00F58375F00DE52B121E9DE4F0052BE52B92
:10355E00B407DF0535E535B408B3E4F53DF525F5DB
:10356E0027F529F533F53CF52BF526F535F532C261
:10357E00ADF5C9D2CDD2CCC2C9C2CAF5CDF5CC906B
:10358E007475E0F5CBA3E0F5CA85CBCD85CACCD258
:10359E009ED29CD2CAC2ACC298C29975B81075B7E9
:0435AE0010D2AC2269
:0100220022BB
:103022008F57300C0EE540B44209E5436402700349
:10303200023136E54154E324DF605624DF60351463
:10304200603224E360681470030230F814700302E3
:10305200311F24E2601E24606003023136E54275AE
:10306200F00DA4242AF582E43461F5837D40AF5744
:103072001229702275F00DE529A424F1F582E5F0FC
:10308200346BF5837D40AF57122970052953293FD0
:103092002275F00DE525A424C9F582E5F03461F529
:1030A200837D40AF57122970052553257F2275F085
:1030B20075E542A42456F582E5F03468F583E543CC
:1030C200543FFF1313543F75F00D121E9D7D40AF08
:1030D2005712297075F068E542A42435F582E5F0AF
:1030E2003471F583E543543FFF1313543F75F00DDC
:1030F200121E9DE4F02275F068E542A42435F582A3
:10310200E5F03471F583E543543FFF1313543F75E3
:10311200F00D121E9D7D40AF571229702275F07579
:10312200E542A42449F582E5F03468F5837D40AF99
:05313200571229702274
:103702008F5A300307906002E04440F090600263F9
:10371200A20190703463A201AF5A122982E4F52EFD
:10372200F52F855A3190703463A20190162363A25B
:1037320001AF31AE30AD2FAC2E1229B58F318E30A4
:103742008D2F8C2E7434255AF582E43470F583E57E
:103752002FF07435255AF582E43470F583E52EF0A6
:103762007434255AF582E43470F583E0F53AA3E027
:10377200F53BE55A2402F52C201B127E147FDD1244
:1037820032437E707F34E4FBAD2C1234067534FF75
:0A379200D202C2992099FDD29922BB
:1007D800301122C211906F33E0600C04F0E0D39422
:1007E800F04004C2AF80FE906194E004F09061C8CC
:1007F800E0600214F0E508B4010CE4F508D202C286
:10080800992099FDD29930020F906194E0D3941405
:10081800400BC202D2108005E4906194F0300621AA
:1008280030970E200507907134E004F528D2058032
:100838001030050A201B077E147FE3123243C205DD
:1008480022907134E0FFE528D39F403C201B077EAF
:10085800147FED123243300E15E4906193F0C20D0F
:10086800C209FF12400C9061C87402F08007E4903E
:1008780061C8F0D209E4F52DF538F52AF528C2014A
:10088800906000F0A3F0D2109061C7E0FF700302FF
:10089800092624FE601C14602514605114605A1443
:1008A800606A24057078201B757E147FFC12324321
:1008B800806C201B697E157F071232438060201BE5
:1008C800077E157F17123243300D53E4906193F081
:1008D800C20DC2099061C8F0F52DF538752A03F5E7
:1008E80028C201906000F0A3F0D2108031201B2EA6
:1008F8007E157F261232438025201B077E157F3404
:10090800123243907134E004F5288012201B077ED0
:10091800157F4C123243907134E004F52822300DD3
:1009280003020A7D9061C8E06003020A7D2010037B
:10093800020A7D906193E014603114606E147003B4
:10094800020A2624036003020A787F0112400C90F1
:100958006193E004F09061C87401F0301B03020A4F
:100968007D7E157F61123243020A7D201B077E15AA
:100978007F6612324378347C707D017BFF7A187968
:1009880023121F71E4F52DF538F5349061C7F00591
:1009980028C201D202C2992099FDD299906193E0B0
:1009A80004F09061C8740AF0020A7D9061C7E0FF04
:1009B800B403119061937403F005289061C8743CE6
:1009C800F0020A7DEF6401601C201B0AEF70077EAD
:1009D800157F721232439061C8740AF09061937463
:1009E80001F0020A7D201B077E157F7F12324378B3
:1009F800347C707D017B017A617902121F71E4F504
:100A08002DF538F534C201D202C2992099FDD29948
:100A1800906193E004F09061C87406F0805790618B
:100A2800C7E0FFB40106A3743CF08049EFB4030AA1
:100A380005289061C8743CF0803BEFB40217E4F5D8
:100A480028D20DD209F52AC20F906000740BF0A3CA
:100A580074B8F08020201B0AEF70077E157F721291
:100A680032439061C8740AF09061937401F0800574
:100A7800E4906193F0E49061C7F0200D03020CE963
:100A8800E532C394144003020CE9E5296527605A4E
:100A980075F00DE527A424F5F582E5F0346BF583B0
:100AA800E02405F557C3940E502E75F00DE527A4E4
:100AB80024F1F582E5F0346BF58363A20174042513
:100AC80032F582E43460F58363A201AF57122982BC
:100AD800E5572532F532800A201B077E157F8812DC
:100AE8003243052753273F020CE975F075E535A415
:100AF8002449F582E5F03468F583E07003020C01BF
:100B0800E526705775F075E535A4244DF582E5F0B6
:100B18003468F583E02405F557C3940E502E75F01C
:100B280075E535A42449F582E5F03468F58363A2B8
:100B38000174042532F582E43460F58363A201AFC1
:100B480057122982E5572532F532800A201B077E85
:100B5800157F881232430526020CE975F075E535D4
:100B6800A4244CF582E5F03468F583E0540FFFE5E2
:100B780026D39F506775F075E535A4244DF582E5B9
:100B8800F03468F58375F00DE526121E9DE0240506
:100B9800F557C3940E503675F075E535A42449F51C
:100BA80082E5F03468F58375F00DE526121E9D6325
:100BB800A20174042532F582E43460F58363A2014E
:100BC800AF57122982E5572532F532800A201B07D4
:100BD8007E157F881232430526020CE9E4F5267556
:100BE800F075E535A42449F582E5F03468F583E429
:100BF800F00535533507020CE90535533507E5256A
:100C0800653D605E053D533D7F75F00DE53DA424CF
:100C1800CDF582E5F03461F583E02405F557C394FA
:100C28000E502F75F00DE53DA424C9F582E5F0348A
:100C380061F58363A20174042532F582E43460F51A
:100C48008363A201AF57122982E5572532F5320294
:100C58000CE9301B03020CE97E157F88123243022F
:100C68000CE9E53375F00DA4242AF582E43461F526
:100C780083E06068E53375F00DA4242EF582E43432
:100C880061F583E02405F557C3940E502DE53375BF
:100C9800F00DA4242AF582E43461F58363A201747B
:100CA800042532F582E43460F58363A201AF57125C
:100CB8002982E5572532F532800A201B077E157FE9
:100CC80088123243E53375F00DA4242AF582E43402
:100CD80061F583E4F0053353330780050533533357
:100CE80007300203020DBDE5086003020DBD200DAB
:100CF80003020DBDE52A6401707B30072820082017
:100D080030030FE532600B200F089060027410F07A
:100D1800801FE4906002F0A37419F07F021237027A
:100D2800C207020DBDE5326028200F25E49060025D
:100D3800F09060037419F0E5322402FF12370205BF
:100D480028200802D20FE4F532906000F0A3F0806A
:100D580064D3906001E094E8906000E0940340550B
:100D6800E4F0A3F0300F4EC20F201B497E157F938D
:100D78001232438040E52A703C200406752A01F5AA
:100D88003222D3906001E094E8906000E094034040
:100D980024E4F0A3F0A374FEF0A374A0F0A374FFFE
:100DA800F07F03123702E4F5320528201B077E1571
:100DB8007FA3123243E5387003020F4BF557E4F571
:100DC80038F52EF52FE557547FF531E55754802433
:100DD80034F582E4346FF58363A20190162363A28D
:100DE80001AF31AE30AD2FAC2E1229B58F318E3018
:100DF8008D2F8C2EE55754802434F582E4346FAF60
:100E080082F5588F5953577F74322557F582E43449
:100E18006FF583E0FEA3E0653B7003EE653A70264C
:100E2800201B077E157FAE123243E52CB5571120E3
:100E38001B077E157FC212324374052528F5282228
:100E480074032528F528E52F452E6022301B030260
:100E58000F4B7E157FCC123243E4FBAD57AF59AE32
:100E6800581234067D03AF2FAE2E12332822201BD2
:100E780018E52A640160127E157FD7123243E4FB1D
:100E8800AD57AF59AE58123406E557B40406E4F529
:100E980028C20F22855982855883A3E024E7603051
:100EA8002499601F24F06003020F41752A01A207EC
:100EB8009207E4F532301B03020F4B7E157FDC12DC
:100EC800324322D207201B7B7E157FE91232432250
:100ED800E52A700B201B6C7E157FF61232432285A3
:100EE8005982855883E030E405E4F528C20FD2071B
:100EF800E55724FCF551201B1A7E167F1612324343
:100F0800E5592402FFE43558FEE55724FCFDE4FBCF
:100F1800123406E551C3940F501BE5592402FFE42F
:100F28003558F5838F8263A201907A8563A201AF59
:100F38005112298222E4F55122201B077E167F1EBA
:030F48001232431F
:010F4B002283
:10383E00020026E493A3F8E493A34003F68001F27A
:10384E0008DFF48029E493A3F85407240CC8C3338B
:10385E00C4540F4420C8834004F456800146F6DF5A
:10386E00E4800B010204081020408090401DE47E8D
:10387E00019360BCA3FF543F30E509541FFEE4934F
:10388E00A360010ECF54C025E060A840B8E493A316
:10389E00FAE493A3F8E493A3C8C582C8CAC583CA41
:1038AE00F0A3C8C582C8CAC583CADFE9DEE780BEF9
:01402300009C
:101D0100BB010689828A83E0225002E722BBFE02E0
:091D1100E32289828A83E4932213
:101D1A00BB010CE58229F582E5833AF583E022507E
:101D2A0006E92582F8E622BBFE06E92582F8E222C8
:0D1D3A00E58229F582E5833AF583E49322E2
:101D4700A3F8E0C5F025F0F0E5821582700215834F
:061D5700E0C838F0E822AC
:101D5D0075F008758200EF2FFFEE33FECD33CDCC3D
:101D6D0033CCC58233C5829BED9AEC99E5829840C0
:101D7D000CF582EE9BFEED9AFDEC99FC0FD5F0D69D
:101D8D00E4CEFBE4CDFAE4CCF9A88222B800C1B9C7
:101D9D000059BA002DEC8BF084CFCECDFCE5F0CB05
:101DAD00F97818EF2FFFEE33FEED33FDEC33FCEB3E
:101DBD0033FB10D703994004EB99FB0FD8E5E4F9F9
:101DCD00FA227818EF2FFFEE33FEED33FDEC33FCE6
:101DDD00C933C910D7059BE99A4007EC9BFCE99ADA
:101DED00F90FD8E0E4C9FAE4CCFB2275F010EF2F1F
:101DFD00FFEE33FEED33FDCC33CCC833C810D7071F
:101E0D009BEC9AE899400AED9BFDEC9AFCE899F859
:0E1E1D000FD5F0DAE4CDFBE4CCFAE4C8F922EC
:0E1E2B00C3E49FFFE49EFEE49DFDE49CFC22C8
:101E3900EB9FF5F0EA9E42F0E99D42F0EC6480C820
:061E490064809845F022C0
:101E4F00EB9FF5F0EA9E42F0E99D42F0E89C45F0E9
:011E5F002260
:0C1E6000ECF0A3EDF0A3EEF0A3EFF022F5
:101E6C00A8828583F0D083D082121E83121E831227
:101E7C001E83121E83E473E493A3C583C5F0C5834C
:101E8C00C8C582C8F0A3C583C5F0C583C8C582C8C0
:011E9C002223
:0C1E9D00A42582F582E5F03583F5832250
:102A59008B568A578958E4F562F561F560F55FF59B
:102A69005DF55EE55A455B45596012EBC0E0EAC089
:102A7900E0E9C0E0AB59AA5AA95B121FDDAB5605C4
:102A890058E558AA577002055714F9121D01F56344
:102A9900C394094007E563D3940D40E1E5636420DD
:102AA90060DBE563B42D05435E038016E563B42B53
:102AB90005435E01800C74FF2558F55874FF35579E
:102AC900F557E55C60046410703FAB56AA57A958E6
:102AD900121D0164306009E55C702E755C0A80295D
:102AE900900001121D1AFF64786004EFB458134373
:102AF9005E01755C1074022558F558E43557F55791
:102B09008007E55C7003755C08AB560558E558AA63
:102B1900577002055714F9121D01F563C3946140FA
:102B29000AE563D3947A50035363DF74D02563F5C0
:102B390063C3940A400CE5639411406D74F92563ED
:102B4900F563E563D3955C5060435E0185626785F3
:102B59006166856065855F64AF5C7E00E4FCFDAB02
:102B690062AA61A960A85F121F8EC8ECC8C9EDC925
:102B7900CAEECACBEFCBE4FCFDFEEB2563F562EEB2
:102B89003AF561ED39F560EC38F55FAF62AE61ADEC
:102B990060FCAB67AA66A965A864D3121E4F5003EF
:102BA900022B12435E04022B12E55E20E003E4804F
:102BB9002DE55A455B4559601EAB56E55824FFF98A
:102BC900E55734FFFAEBC0E0EAC0E0E9C0E0AB59F1
:102BD900AA5AA95B121FDDE55E30E20774FFFFFE0A
:102BE900FDFC22E55EAF62AE61AD60AC5F30E10332
:042BF900021E2B226B
:101EA900E709F60870FA8046E709F20870FA803EF9
:101EB90088828C83E709F0A370FA807CE309F6082D
:101EC90070FA8074E309F20870FA806C88828C8356
:101ED900E309F0A370FA806089828A83E0A3F60897
:101EE90070FA805489828A83E0A3F20870FA8048E4
:101EF90080D280FA80C680D4806180F2802F8010E1
:101F090080A680EA809A80A880DA80E280CA802F41
:101F190089828A8363A20188828C8363A201E49304
:101F2900A363A201F0A363A20170F3800B89828AE3
:101F390083E493A3F60870F9ECFAA9F0EDFB228982
:101F4900828A8363A20188828C8363A201E0A363EE
:101F5900A201F0A363A20170F480DD89828A83E47F
:101F690093A3F20870F980D088F0ED2402B404003C
:101F790050C6F582EB2402B4040050BC23234582E9
:051F890023901EF97316
:101F8E00E88FF0A4CC8BF0A42CFCE98EF0A42CFCF2
:101F9E008AF0EDA42CFCEA8EF0A4CDA8F08BF0A470
:101FAE002DCC3825F0FDE98FF0A42CCD35F0FCEBCF
:101FBE008EF0A4FEA9F0EB8FF0A4CFC5F02ECD3994
:0F1FCE00FEE43CFCEAA42DCE35F0FDE43CFC2201
:101FDD00BB011A89828A83D0F0D0E0F8D0E0F9D025
:101FED00E0FAD0E0FBE8C0E0C0F00220355016E981
:101FFD00F8D083D082D0E0F9D0E0FAD0E0FBC082F7
:10200D00C08302202CBBFE16E9F8D083D082D0E02D
:0F201D00F9D0E0FAD0E0FBC082C08302203E225F
:09202C00EBF608EAF608E9F622D9
:09203500EBF0A3EAF0A3E9F022AC
:09203E00EBF208EAF208E9F222D3
:00000001FF
